 Half_dll_d

 Timestamp is 44d97e3d (Tue Aug 08 23:18:37 2006)

 Preferred load address is 10000000

 Start         Length     Name                   Class
 0001:00000000 00004252H .text                   CODE
 0001:00004260 0000108eH .text$x                 CODE
 0002:00000000 00000104H .CRT$XCA                DATA
 0002:00000104 00000104H .CRT$XCZ                DATA
 0002:00000208 00000104H .CRT$XIA                DATA
 0002:0000030c 00000104H .CRT$XIAA               DATA
 0002:00000410 00000104H .CRT$XIZ                DATA
 0002:00000520 00000c28H .rdata                  DATA
 0002:00001148 00000155H .rdata$debug            DATA
 0002:000012a0 00000113H .rdata$sxdata           DATA
 0002:000013b4 00000104H .rtc$IAA                DATA
 0002:000014b8 00000104H .rtc$IMZ                DATA
 0002:000015bc 00000104H .rtc$IZZ                DATA
 0002:000016c0 00000104H .rtc$TAA                DATA
 0002:000017c4 00000104H .rtc$TMZ                DATA
 0002:000018c8 00000104H .rtc$TZZ                DATA
 0002:000019d0 000002aaH .xdata$x                DATA
 0002:00001c80 0000018bH .edata                  DATA
 0003:00000000 0004d317H .data                   DATA
 0003:0004d318 00000390H .bss                    DATA
 0004:00000000 0000003cH .idata$2                DATA
 0004:0000003c 00000014H .idata$3                DATA
 0004:00000050 000001bcH .idata$4                DATA
 0004:0000020c 000001bcH .idata$5                DATA
 0004:000003c8 0000095aH .idata$6                DATA

  Address         Publics by Value              Rva+Base       Lib:Object

 0000:00000000       __except_list              00000000     <absolute>
 0000:00000004       ___safe_se_handler_count   00000004     <absolute>
 0000:00009876       __ldused                   00009876     <absolute>
 0000:00009876       __fltused                  00009876     <absolute>
 0000:00000000       ___ImageBase               10000000     <linker-defined>
 0001:000000c0       ?overflow@half@@CAMXZ      100010c0 f   half.obj
 0001:00000110       ?convert@half@@CAFH@Z      10001110 f   half.obj
 0001:00000250       ??6@YAAAV?$basic_ostream@DU?$char_traits@D@std@@@std@@AAV01@Vhalf@@@Z 10001250 f   half.obj
 0001:00000280       ??5@YAAAV?$basic_istream@DU?$char_traits@D@std@@@std@@AAV01@AAVhalf@@@Z 10001280 f   half.obj
 0001:00000310       ?printBits@@YAXAAV?$basic_ostream@DU?$char_traits@D@std@@@std@@Vhalf@@@Z 10001310 f   half.obj
 0001:00000390       ?printBits@@YAXAAV?$basic_ostream@DU?$char_traits@D@std@@@std@@M@Z 10001390 f   half.obj
 0001:00000440       ?printBits@@YAXQADVhalf@@@Z 10001440 f   half.obj
 0001:000004e0       ?printBits@@YAXQADM@Z      100014e0 f   half.obj
 0001:000006d0       ??Bhalf@@QBEMXZ            100016d0 f i half.obj
 0001:00000700       ??0half@@QAE@M@Z           10001700 f i half.obj
 0001:00000800       ??4half@@QAEAAV0@V0@@Z     10001800 f i half.obj
 0001:00000830       ?bits@half@@QBEGXZ         10001830 f i half.obj
 0001:00000850       ??$?6U?$char_traits@D@std@@@std@@YAAAV?$basic_ostream@DU?$char_traits@D@std@@@0@AAV10@D@Z 10001850 f i half.obj
 0001:00000d10       ??0sentry@?$basic_ostream@DU?$char_traits@D@std@@@std@@QAE@AAV12@@Z 10001d10 f i half.obj
 0001:00000e50       ??1sentry@?$basic_ostream@DU?$char_traits@D@std@@@std@@QAE@XZ 10001e50 f i half.obj
 0001:00000f00       ??Bsentry@?$basic_ostream@DU?$char_traits@D@std@@@std@@QBE_NXZ 10001f00 f i half.obj
 0001:00000f20       ??0_Sentry_base@?$basic_ostream@DU?$char_traits@D@std@@@std@@QAE@AAV12@@Z 10001f20 f i half.obj
 0001:00000fc0       ??1_Sentry_base@?$basic_ostream@DU?$char_traits@D@std@@@std@@QAE@XZ 10001fc0 f i half.obj
 0001:0000104a       ??6?$basic_ostream@DU?$char_traits@D@std@@@std@@QAEAAV01@M@Z 1000204a f   msvcprtd:MSVCP80D.dll
 0001:00001050       ??5?$basic_istream@DU?$char_traits@D@std@@@std@@QAEAAV01@AAM@Z 10002050 f   msvcprtd:MSVCP80D.dll
 0001:00001056       ?width@ios_base@std@@QAEHH@Z 10002056 f   msvcprtd:MSVCP80D.dll
 0001:0000105c       ?setstate@?$basic_ios@DU?$char_traits@D@std@@@std@@QAEXH_N@Z 1000205c f   msvcprtd:MSVCP80D.dll
 0001:00001062       ?eq_int_type@?$char_traits@D@std@@SA_NABH0@Z 10002062 f   msvcprtd:MSVCP80D.dll
 0001:00001068       ?eof@?$char_traits@D@std@@SAHXZ 10002068 f   msvcprtd:MSVCP80D.dll
 0001:0000106e       ?sputc@?$basic_streambuf@DU?$char_traits@D@std@@@std@@QAEHD@Z 1000206e f   msvcprtd:MSVCP80D.dll
 0001:00001074       ?rdbuf@?$basic_ios@DU?$char_traits@D@std@@@std@@QBEPAV?$basic_streambuf@DU?$char_traits@D@std@@@2@XZ 10002074 f   msvcprtd:MSVCP80D.dll
 0001:0000107a       ?fill@?$basic_ios@DU?$char_traits@D@std@@@std@@QBEDXZ 1000207a f   msvcprtd:MSVCP80D.dll
 0001:00001080       ?flags@ios_base@std@@QBEHXZ 10002080 f   msvcprtd:MSVCP80D.dll
 0001:00001086       ?width@ios_base@std@@QBEHXZ 10002086 f   msvcprtd:MSVCP80D.dll
 0001:0000108c       ?flush@?$basic_ostream@DU?$char_traits@D@std@@@std@@QAEAAV12@XZ 1000208c f   msvcprtd:MSVCP80D.dll
 0001:00001092       ?tie@?$basic_ios@DU?$char_traits@D@std@@@std@@QBEPAV?$basic_ostream@DU?$char_traits@D@std@@@2@XZ 10002092 f   msvcprtd:MSVCP80D.dll
 0001:00001098       ?good@ios_base@std@@QBE_NXZ 10002098 f   msvcprtd:MSVCP80D.dll
 0001:0000109e       ?_Osfx@?$basic_ostream@DU?$char_traits@D@std@@@std@@QAEXXZ 1000209e f   msvcprtd:MSVCP80D.dll
 0001:000010a4       ?uncaught_exception@std@@YA_NXZ 100020a4 f   msvcprtd:MSVCP80D.dll
 0001:000010aa       ?_Lock@?$basic_streambuf@DU?$char_traits@D@std@@@std@@QAEXXZ 100020aa f   msvcprtd:MSVCP80D.dll
 0001:000010b0       ?_Unlock@?$basic_streambuf@DU?$char_traits@D@std@@@std@@QAEXXZ 100020b0 f   msvcprtd:MSVCP80D.dll
 0001:000010c0       __RTC_InitBase             100020c0 f   MSVCRTD:init.obj
 0001:000010f0       __RTC_Shutdown             100020f0 f   MSVCRTD:init.obj
 0001:00001110       __RTC_CheckEsp             10002110 f   MSVCRTD:stack.obj
 0001:00001140       @_RTC_CheckStackVars@8     10002140 f   MSVCRTD:stack.obj
 0001:000011a0       @_RTC_AllocaHelper@12      100021a0 f   MSVCRTD:stack.obj
 0001:000011d0       @_RTC_CheckStackVars2@12   100021d0 f   MSVCRTD:stack.obj
 0001:000012a6       ___CxxFrameHandler3        100022a6 f   MSVCRTD:MSVCR80D.dll
 0001:000012b0       @__security_check_cookie@4 100022b0 f   MSVCRTD:secchk.obj
 0001:00001340       __CRT_INIT@12              10002340 f   MSVCRTD:crtdll.obj
 0001:00001570       _NtCurrentTeb              10002570 f i MSVCRTD:crtdll.obj
 0001:00001580       __DllMainCRTStartup@12     10002580 f   MSVCRTD:crtdll.obj
 0001:00001770       __RTC_NumErrors            10002770 f   MSVCRTD:userapi.obj
 0001:00001780       __RTC_GetErrDesc           10002780 f   MSVCRTD:userapi.obj
 0001:000017a0       __RTC_SetErrorType         100027a0 f   MSVCRTD:userapi.obj
 0001:000017d0       __RTC_SetErrorFunc         100027d0 f   MSVCRTD:userapi.obj
 0001:000017f0       __RTC_SetErrorFuncW        100027f0 f   MSVCRTD:userapi.obj
 0001:00001810       ?_RTC_GetErrorFunc@@YAP6AHHPBDH00ZZPBX@Z 10002810 f   MSVCRTD:userapi.obj
 0001:00001820       ?_RTC_GetErrorFuncW@@YAP6AHHPB_WH00ZZPBX@Z 10002820 f   MSVCRTD:userapi.obj
 0001:00001826       __CRT_RTC_INITW            10002826 f   MSVCRTD:MSVCR80D.dll
 0001:00001830       _DebuggerKnownHandle       10002830 f   MSVCRTD:error.obj
 0001:000018d0       ?_RTC_Failure@@YAXPAXH@Z   100028d0 f   MSVCRTD:error.obj
 0001:00001c00       ?_RTC_StackFailure@@YAXPAXPBD@Z 10002c00 f   MSVCRTD:error.obj
 0001:00001d20       ?_RTC_AllocaFailure@@YAXPAXPAU_RTC_ALLOCA_NODE@@H@Z 10002d20 f   MSVCRTD:error.obj
 0001:00001ee0       __RTC_UninitUse            10002ee0 f   MSVCRTD:error.obj
 0001:00001ff0       ___report_gsfailure        10002ff0 f   MSVCRTD:gs_report.obj
 0001:00002100       ___clean_type_info_names   10003100 f   MSVCRTD:tncleanup.obj
 0001:00002120       __onexit                   10003120 f   MSVCRTD:atonexit.obj
 0001:00002220       _atexit                    10003220 f   MSVCRTD:atonexit.obj
 0001:00002240       __RTC_Initialize           10003240 f   MSVCRTD:initsect.obj
 0001:00002270       __RTC_Terminate            10003270 f   MSVCRTD:initsect.obj
 0001:00002296       __encode_pointer           10003296 f   MSVCRTD:MSVCR80D.dll
 0001:0000229c       __malloc_dbg               1000329c f   MSVCRTD:MSVCR80D.dll
 0001:000022a2       __encoded_null             100032a2 f   MSVCRTD:MSVCR80D.dll
 0001:000022a8       __free_dbg                 100032a8 f   MSVCRTD:MSVCR80D.dll
 0001:000022ae       __decode_pointer           100032ae f   MSVCRTD:MSVCR80D.dll
 0001:000022b4       __CrtSetCheckCount         100032b4 f   MSVCRTD:MSVCR80D.dll
 0001:000022c0       __ValidateImageBase        100032c0 f   MSVCRTD:pesect.obj
 0001:00002320       __FindPESection            10003320 f   MSVCRTD:pesect.obj
 0001:000023a0       __IsNonwritableInCurrentImage 100033a0 f   MSVCRTD:pesect.obj
 0001:000024b0       __initterm                 100034b0 f   MSVCRTD:MSVCR80D.dll
 0001:000024b6       __initterm_e               100034b6 f   MSVCRTD:MSVCR80D.dll
 0001:000024bc       __amsg_exit                100034bc f   MSVCRTD:MSVCR80D.dll
 0001:000024d0       ___security_init_cookie    100034d0 f   MSVCRTD:gs_support.obj
 0001:000025ea       ___CppXcptFilter           100035ea f   MSVCRTD:MSVCR80D.dll
 0001:000025f0       _DllMain@12                100035f0 f   MSVCRTD:dllmain.obj
 0001:00002620       __except_handler4          10003620 f   MSVCRTD:chandler4gs.obj
 0001:00002650       ?_RTC_GetSrcLine@@YAHPAEPA_WKPAH1K@Z 10003650 f   MSVCRTD:pdblkup.obj
 0001:00002adc       __crt_debugger_hook        10003adc f   MSVCRTD:MSVCR80D.dll
 0001:00002ae2       ___clean_type_info_names_internal 10003ae2 f   MSVCRTD:MSVCR80D.dll
 0001:00002ae8       __unlock                   10003ae8 f   MSVCRTD:MSVCR80D.dll
 0001:00002aee       ___dllonexit               10003aee f   MSVCRTD:MSVCR80D.dll
 0001:00002af4       __lock                     10003af4 f   MSVCRTD:MSVCR80D.dll
 0001:00002afa       __except_handler4_common   10003afa f   MSVCRTD:MSVCR80D.dll
 0001:00002b00       _InterlockedExchange@8     10003b00 f   kernel32:KERNEL32.dll
 0001:00002b06       _Sleep@4                   10003b06 f   kernel32:KERNEL32.dll
 0001:00002b0c       _InterlockedCompareExchange@12 10003b0c f   kernel32:KERNEL32.dll
 0001:00002b12       _RaiseException@16         10003b12 f   kernel32:KERNEL32.dll
 0001:00002b18       _DebugBreak@0              10003b18 f   kernel32:KERNEL32.dll
 0001:00002b1e       _WideCharToMultiByte@32    10003b1e f   kernel32:KERNEL32.dll
 0001:00002b24       _IsDebuggerPresent@0       10003b24 f   kernel32:KERNEL32.dll
 0001:00002b2a       _MultiByteToWideChar@24    10003b2a f   kernel32:KERNEL32.dll
 0001:00002b30       _lstrlenA@4                10003b30 f   kernel32:KERNEL32.dll
 0001:00002b36       _GetProcAddress@8          10003b36 f   kernel32:KERNEL32.dll
 0001:00002b3c       _LoadLibraryA@4            10003b3c f   kernel32:KERNEL32.dll
 0001:00002b42       _TerminateProcess@8        10003b42 f   kernel32:KERNEL32.dll
 0001:00002b48       _GetCurrentProcess@0       10003b48 f   kernel32:KERNEL32.dll
 0001:00002b4e       _UnhandledExceptionFilter@4 10003b4e f   kernel32:KERNEL32.dll
 0001:00002b54       _SetUnhandledExceptionFilter@4 10003b54 f   kernel32:KERNEL32.dll
 0001:00002b5a       _QueryPerformanceCounter@4 10003b5a f   kernel32:KERNEL32.dll
 0001:00002b60       _GetTickCount@0            10003b60 f   kernel32:KERNEL32.dll
 0001:00002b66       _GetCurrentThreadId@0      10003b66 f   kernel32:KERNEL32.dll
 0001:00002b6c       _GetCurrentProcessId@0     10003b6c f   kernel32:KERNEL32.dll
 0001:00002b72       _GetSystemTimeAsFileTime@4 10003b72 f   kernel32:KERNEL32.dll
 0001:00002b78       _FatalAppExitA@8           10003b78 f   kernel32:KERNEL32.dll
 0001:00002b7e       _DisableThreadLibraryCalls@4 10003b7e f   kernel32:KERNEL32.dll
 0001:00002b84       _HeapFree@12               10003b84 f   kernel32:KERNEL32.dll
 0001:00002b8a       _HeapAlloc@12              10003b8a f   kernel32:KERNEL32.dll
 0001:00002b90       _GetProcessHeap@0          10003b90 f   kernel32:KERNEL32.dll
 0001:00002b96       _GetModuleFileNameW@12     10003b96 f   kernel32:KERNEL32.dll
 0001:00002b9c       _VirtualQuery@12           10003b9c f   kernel32:KERNEL32.dll
 0001:00002ba2       _FreeLibrary@4             10003ba2 f   kernel32:KERNEL32.dll
 0002:00000000       ___xc_a                    10007000     MSVCRTD:cinitexe.obj
 0002:00000104       ___xc_z                    10007104     MSVCRTD:cinitexe.obj
 0002:00000208       ___xi_a                    10007208     MSVCRTD:cinitexe.obj
 0002:00000410       ___xi_z                    10007410     MSVCRTD:cinitexe.obj
 0002:00000550       ?collate@?$_Locbase@H@std@@2HB 10007550     half.obj
 0002:00000554       ?ctype@?$_Locbase@H@std@@2HB 10007554     half.obj
 0002:00000558       ?monetary@?$_Locbase@H@std@@2HB 10007558     half.obj
 0002:0000055c       ?numeric@?$_Locbase@H@std@@2HB 1000755c     half.obj
 0002:00000560       ?time@?$_Locbase@H@std@@2HB 10007560     half.obj
 0002:00000564       ?messages@?$_Locbase@H@std@@2HB 10007564     half.obj
 0002:00000568       ?all@?$_Locbase@H@std@@2HB 10007568     half.obj
 0002:0000056c       ?none@?$_Locbase@H@std@@2HB 1000756c     half.obj
 0002:00000570       ?skipws@?$_Iosb@H@std@@2W4_Fmtflags@12@B 10007570     half.obj
 0002:00000574       ?unitbuf@?$_Iosb@H@std@@2W4_Fmtflags@12@B 10007574     half.obj
 0002:00000578       ?uppercase@?$_Iosb@H@std@@2W4_Fmtflags@12@B 10007578     half.obj
 0002:0000057c       ?showbase@?$_Iosb@H@std@@2W4_Fmtflags@12@B 1000757c     half.obj
 0002:00000580       ?showpoint@?$_Iosb@H@std@@2W4_Fmtflags@12@B 10007580     half.obj
 0002:00000584       ?showpos@?$_Iosb@H@std@@2W4_Fmtflags@12@B 10007584     half.obj
 0002:00000588       ?left@?$_Iosb@H@std@@2W4_Fmtflags@12@B 10007588     half.obj
 0002:0000058c       ?right@?$_Iosb@H@std@@2W4_Fmtflags@12@B 1000758c     half.obj
 0002:00000590       ?internal@?$_Iosb@H@std@@2W4_Fmtflags@12@B 10007590     half.obj
 0002:00000594       ?dec@?$_Iosb@H@std@@2W4_Fmtflags@12@B 10007594     half.obj
 0002:00000598       ?oct@?$_Iosb@H@std@@2W4_Fmtflags@12@B 10007598     half.obj
 0002:0000059c       ?hex@?$_Iosb@H@std@@2W4_Fmtflags@12@B 1000759c     half.obj
 0002:000005a0       ?scientific@?$_Iosb@H@std@@2W4_Fmtflags@12@B 100075a0     half.obj
 0002:000005a4       ?fixed@?$_Iosb@H@std@@2W4_Fmtflags@12@B 100075a4     half.obj
 0002:000005a8       ?boolalpha@?$_Iosb@H@std@@2W4_Fmtflags@12@B 100075a8     half.obj
 0002:000005ac       ?_Stdio@?$_Iosb@H@std@@2W4_Fmtflags@12@B 100075ac     half.obj
 0002:000005b0       ?adjustfield@?$_Iosb@H@std@@2W4_Fmtflags@12@B 100075b0     half.obj
 0002:000005b4       ?basefield@?$_Iosb@H@std@@2W4_Fmtflags@12@B 100075b4     half.obj
 0002:000005b8       ?floatfield@?$_Iosb@H@std@@2W4_Fmtflags@12@B 100075b8     half.obj
 0002:000005bc       ?goodbit@?$_Iosb@H@std@@2W4_Iostate@12@B 100075bc     half.obj
 0002:000005c0       ?eofbit@?$_Iosb@H@std@@2W4_Iostate@12@B 100075c0     half.obj
 0002:000005c4       ?failbit@?$_Iosb@H@std@@2W4_Iostate@12@B 100075c4     half.obj
 0002:000005c8       ?badbit@?$_Iosb@H@std@@2W4_Iostate@12@B 100075c8     half.obj
 0002:000005cc       ?_Hardfail@?$_Iosb@H@std@@2W4_Iostate@12@B 100075cc     half.obj
 0002:000005d0       ?in@?$_Iosb@H@std@@2W4_Openmode@12@B 100075d0     half.obj
 0002:000005d4       ?out@?$_Iosb@H@std@@2W4_Openmode@12@B 100075d4     half.obj
 0002:000005d8       ?ate@?$_Iosb@H@std@@2W4_Openmode@12@B 100075d8     half.obj
 0002:000005dc       ?app@?$_Iosb@H@std@@2W4_Openmode@12@B 100075dc     half.obj
 0002:000005e0       ?trunc@?$_Iosb@H@std@@2W4_Openmode@12@B 100075e0     half.obj
 0002:000005e4       ?_Nocreate@?$_Iosb@H@std@@2W4_Openmode@12@B 100075e4     half.obj
 0002:000005e8       ?_Noreplace@?$_Iosb@H@std@@2W4_Openmode@12@B 100075e8     half.obj
 0002:000005ec       ?binary@?$_Iosb@H@std@@2W4_Openmode@12@B 100075ec     half.obj
 0002:000005f0       ?beg@?$_Iosb@H@std@@2W4_Seekdir@12@B 100075f0     half.obj
 0002:000005f4       ?cur@?$_Iosb@H@std@@2W4_Seekdir@12@B 100075f4     half.obj
 0002:000005f8       ?end@?$_Iosb@H@std@@2W4_Seekdir@12@B 100075f8     half.obj
 0002:000005fc       __real@501502f9            100075fc     half.obj
 0002:00000600       __real@0000000000000000    10007600     half.obj
 0002:0000060c       __pDefaultRawDllMain       1000760c     MSVCRTD:crtdll.obj
 0002:0000060c       __pRawDllMain              1000760c     MSVCRTD:crtdll.obj
 0002:00000610       ??_C@_08EIBOPINA@crtdll?4c?$AA@ 10007610     MSVCRTD:crtdll.obj
 0002:0000061c       ??_C@_0BP@OGBCLIBO@Stack?5around?5_alloca?5corrupted?$AA@ 1000761c     MSVCRTD:userapi.obj
 0002:0000063c       ??_C@_0CK@CNLNOEPB@Local?5variable?5used?5before?5initi@ 1000763c     MSVCRTD:userapi.obj
 0002:00000668       ??_C@_0BI@CIGMDCBH@Stack?5memory?5corruption?$AA@ 10007668     MSVCRTD:userapi.obj
 0002:00000680       ??_C@_0CK@FEGOIOPB@Cast?5to?5smaller?5type?5causing?5los@ 10007680     MSVCRTD:userapi.obj
 0002:000006ac       ??_C@_0BJ@HEGAHDFO@Stack?5pointer?5corruption?$AA@ 100076ac     MSVCRTD:userapi.obj
 0002:000006c8       ??_C@_0BO@GNIAFIKK@Unknown?5Runtime?5Check?5Error?6?$AN?$AA@ 100076c8     MSVCRTD:error.obj
 0002:000006e8       ??_C@_0CM@NGINOKPC@Stack?5memory?5around?5_alloca?5was?5@ 100076e8     MSVCRTD:error.obj
 0002:00000714       ??_C@_0DG@HKJMLLLP@A?5local?5variable?5was?5used?5before@ 10007714     MSVCRTD:error.obj
 0002:0000074c       ??_C@_0BN@FFOINMNJ@Stack?5memory?5was?5corrupted?6?$AN?$AA@ 1000774c     MSVCRTD:error.obj
 0002:00000770       ??_C@_0BBN@GPMLNJCF@A?5cast?5to?5a?5smaller?5data?5type?5ha@ 10007770     MSVCRTD:error.obj
 0002:00000890       ??_C@_0NN@NGPKDKPD@The?5value?5of?5ESP?5was?5not?5properl@ 10007890     MSVCRTD:error.obj
 0002:000009f0       ??_C@_0CA@IODNCDPG@Run?9Time?5Check?5Failure?5?$CD?$CFd?5?9?5?$CFs?$AA@ 100079f0     MSVCRTD:error.obj
 0002:00000a10       ??_C@_0BE@GNBOBNCK@Unknown?5Module?5Name?$AA@ 10007a10     MSVCRTD:error.obj
 0002:00000a24       ??_C@_0BB@PFFGGCJP@Unknown?5Filename?$AA@ 10007a24     MSVCRTD:error.obj
 0002:00000a38       ??_C@_1EA@NFKNIFJP@?$AAR?$AAu?$AAn?$AA?9?$AAT?$AAi?$AAm?$AAe?$AA?5?$AAC?$AAh?$AAe?$AAc?$AAk?$AA?5?$AAF?$AAa?$AAi?$AAl?$AAu?$AAr?$AAe?$AA?5?$AA?$CD?$AA?$CF?$AAd?$AA?5?$AA?9?$AA?5?$AA?$CF?$AAs?$AA?$AA@ 10007a38     MSVCRTD:error.obj
 0002:00000a78       ??_C@_1GM@OLMCBDMB@?$AAR?$AAu?$AAn?$AAt?$AAi?$AAm?$AAe?$AA?5?$AAC?$AAh?$AAe?$AAc?$AAk?$AA?5?$AAE?$AAr?$AAr?$AAo?$AAr?$AA?4?$AA?6?$AA?$AN?$AA?5?$AAU?$AAn?$AAa?$AAb?$AAl?$AAe?$AA?5?$AAt?$AAo@ 10007a78     MSVCRTD:error.obj
 0002:00000ae4       ??_C@_0CG@IAFNJNEE@Stack?5corrupted?5near?5unknown?5var@ 10007ae4     MSVCRTD:error.obj
 0002:00000b10       ??_C@_0EJ@LJKNEOLN@Stack?5area?5around?5_alloca?5memory@ 10007b10     MSVCRTD:error.obj
 0002:00000b5c       ??_C@_08KJEDNCKC@?$CFs?$CFs?$CFs?$CFs?$AA@ 10007b5c     MSVCRTD:error.obj
 0002:00000b68       ??_C@_02LLMPMKNF@?$DO?5?$AA@ 10007b68     MSVCRTD:error.obj
 0002:00000b6c       ??_C@_01EEMJAFIK@?6?$AA@   10007b6c     MSVCRTD:error.obj
 0002:00000b70       ??_C@_0BC@KIBAILCI@?$CFs?$CFs?$CFp?$CFs?$CFld?$CFs?$CFd?$CFs?$AA@ 10007b70     MSVCRTD:error.obj
 0002:00000b88       ??_C@_0EI@CLEPFNGI@Stack?5area?5around?5_alloca?5memory@ 10007b88     MSVCRTD:error.obj
 0002:00000bd0       ??_C@_0N@MHFFIMFG@?6Address?3?50x?$AA@ 10007bd0     MSVCRTD:error.obj
 0002:00000be0       ??_C@_07DFDJCKFN@?6Size?3?5?$AA@ 10007be0     MSVCRTD:error.obj
 0002:00000be8       ??_C@_0CK@DKGBICFE@?6Allocation?5number?5within?5this?5f@ 10007be8     MSVCRTD:error.obj
 0002:00000c14       ??_C@_08OMAHNMHJ@?6Data?3?5?$DM?$AA@ 10007c14     MSVCRTD:error.obj
 0002:00000c20       ??_C@_09FOPFMPEJ@wsprintfA?$AA@ 10007c20     MSVCRTD:error.obj
 0002:00000c2c       ??_C@_0L@GMPLCCII@user32?4dll?$AA@ 10007c2c     MSVCRTD:error.obj
 0002:00000c38       ??_C@_05MKKEDADM@?$CF?42X?5?$AA@ 10007c38     MSVCRTD:error.obj
 0002:00000c40       ??_C@_0DA@BEGFPCGG@A?5variable?5is?5being?5used?5without@ 10007c40     MSVCRTD:error.obj
 0002:00000c78       ?ProcessDetach@NativeDll@<CrtImplementationDetails>@@0IB 10007c78     MSVCRTD:tncleanup.obj
 0002:00000c7c       ?ProcessAttach@NativeDll@<CrtImplementationDetails>@@0IB 10007c7c     MSVCRTD:tncleanup.obj
 0002:00000c80       ?ThreadAttach@NativeDll@<CrtImplementationDetails>@@0IB 10007c80     MSVCRTD:tncleanup.obj
 0002:00000c84       ?ThreadDetach@NativeDll@<CrtImplementationDetails>@@0IB 10007c84     MSVCRTD:tncleanup.obj
 0002:00000c88       ?ProcessVerifier@NativeDll@<CrtImplementationDetails>@@0IB 10007c88     MSVCRTD:tncleanup.obj
 0002:00000c90       ??_C@_0OH@IHEJDJAH@Microsoft?5Visual?5C?$CL?$CL?5Runtime?5Lib@ 10007c90     MSVCRTD:gs_support.obj
 0002:00000d78       ??_C@_0M@EKFFODEC@MSPDB80?4DLL?$AA@ 10007d78     MSVCRTD:pdblkup.obj
 0002:00000d84       ??_C@_01KDCPPGHE@r?$AA@    10007d84     MSVCRTD:pdblkup.obj
 0002:00000d88       ??_C@_0BB@KCIACLNC@PDBOpenValidate5?$AA@ 10007d88     MSVCRTD:pdblkup.obj
 0002:00000d9c       ??_C@_0BF@BMIHBHCA@EnvironmentDirectory?$AA@ 10007d9c     MSVCRTD:pdblkup.obj
 0002:00000db4       ??_C@_0CN@EAEOKKOC@SOFTWARE?2Microsoft?2VisualStudio?2@ 10007db4     MSVCRTD:pdblkup.obj
 0002:00000de4       ??_C@_0M@HLOHPNFA@RegCloseKey?$AA@ 10007de4     MSVCRTD:pdblkup.obj
 0002:00000df0       ??_C@_0BB@HHEIPGME@RegQueryValueExA?$AA@ 10007df0     MSVCRTD:pdblkup.obj
 0002:00000e04       ??_C@_0O@DCOGKJGG@RegOpenKeyExA?$AA@ 10007e04     MSVCRTD:pdblkup.obj
 0002:00000e14       ??_C@_0N@JJPEKNFO@ADVAPI32?4DLL?$AA@ 10007e14     MSVCRTD:pdblkup.obj
 0002:00000e28       __load_config_used         10007e28     MSVCRTD:loadcfg.obj
 0002:000012a0       ___safe_se_handler_table   100082a0     <linker-defined>
 0002:000013b4       ___rtc_iaa                 100083b4     MSVCRTD:initsect.obj
 0002:000015bc       ___rtc_izz                 100085bc     MSVCRTD:initsect.obj
 0002:000016c0       ___rtc_taa                 100086c0     MSVCRTD:initsect.obj
 0002:000018c8       ___rtc_tzz                 100088c8     MSVCRTD:initsect.obj
 0003:00000008       ?_toFloat@@3PATuif@half@@A 10009008     half.obj
 0003:00040008       ?_eLut@@3PAGA              10049008     half.obj
 0003:0004d1b0       ___security_cookie         100561b0     MSVCRTD:gs_cookie.obj
 0003:0004d1b4       ___security_cookie_complement 100561b4     MSVCRTD:gs_cookie.obj
 0003:0004d1cc       ?_RTC_ErrorLevels@@3PAHA   100561cc     MSVCRTD:error.obj
 0003:0004d1f8       ___native_dllmain_reason   100561f8     MSVCRTD:natstart.obj
 0003:0004d1fc       ___native_vcclrit_reason   100561fc     MSVCRTD:natstart.obj
 0003:0004d328       ?wsprintffp@@3P6AHPADPBDZZA 10056328     MSVCRTD:error.obj
 0003:0004d654       ?__type_info_root_node@@3U__type_info_node@@A 10056654     MSVCRTD:tncleanup.obj
 0003:0004d668       __adjust_fdiv              10056668     <common>
 0003:0004d674       ___native_startup_state    10056674     <common>
 0003:0004d684       ___native_startup_lock     10056684     <common>
 0003:0004d688       ___onexitend               10056688     <common>
 0003:0004d698       ___onexitbegin             10056698     <common>
 0003:0004d69c       ___dyn_tls_init_callback   1005669c     <common>
 0004:00000000       __IMPORT_DESCRIPTOR_MSVCP80D 10057000     msvcprtd:MSVCP80D.dll
 0004:00000014       __IMPORT_DESCRIPTOR_MSVCR80D 10057014     MSVCRTD:MSVCR80D.dll
 0004:00000028       __IMPORT_DESCRIPTOR_KERNEL32 10057028     kernel32:KERNEL32.dll
 0004:0000003c       __NULL_IMPORT_DESCRIPTOR   1005703c     msvcprtd:MSVCP80D.dll
 0004:0000020c       __imp__IsDebuggerPresent@0 1005720c     kernel32:KERNEL32.dll
 0004:00000210       __imp__WideCharToMultiByte@32 10057210     kernel32:KERNEL32.dll
 0004:00000214       __imp__DebugBreak@0        10057214     kernel32:KERNEL32.dll
 0004:00000218       __imp__RaiseException@16   10057218     kernel32:KERNEL32.dll
 0004:0000021c       __imp__InterlockedCompareExchange@12 1005721c     kernel32:KERNEL32.dll
 0004:00000220       __imp__Sleep@4             10057220     kernel32:KERNEL32.dll
 0004:00000224       __imp__InterlockedExchange@8 10057224     kernel32:KERNEL32.dll
 0004:00000228       __imp__lstrlenA@4          10057228     kernel32:KERNEL32.dll
 0004:0000022c       __imp__GetProcAddress@8    1005722c     kernel32:KERNEL32.dll
 0004:00000230       __imp__LoadLibraryA@4      10057230     kernel32:KERNEL32.dll
 0004:00000234       __imp__TerminateProcess@8  10057234     kernel32:KERNEL32.dll
 0004:00000238       __imp__GetCurrentProcess@0 10057238     kernel32:KERNEL32.dll
 0004:0000023c       __imp__UnhandledExceptionFilter@4 1005723c     kernel32:KERNEL32.dll
 0004:00000240       __imp__SetUnhandledExceptionFilter@4 10057240     kernel32:KERNEL32.dll
 0004:00000244       __imp__QueryPerformanceCounter@4 10057244     kernel32:KERNEL32.dll
 0004:00000248       __imp__GetTickCount@0      10057248     kernel32:KERNEL32.dll
 0004:0000024c       __imp__GetCurrentThreadId@0 1005724c     kernel32:KERNEL32.dll
 0004:00000250       __imp__GetCurrentProcessId@0 10057250     kernel32:KERNEL32.dll
 0004:00000254       __imp__FreeLibrary@4       10057254     kernel32:KERNEL32.dll
 0004:00000258       __imp__VirtualQuery@12     10057258     kernel32:KERNEL32.dll
 0004:0000025c       __imp__GetModuleFileNameW@12 1005725c     kernel32:KERNEL32.dll
 0004:00000260       __imp__GetProcessHeap@0    10057260     kernel32:KERNEL32.dll
 0004:00000264       __imp__HeapAlloc@12        10057264     kernel32:KERNEL32.dll
 0004:00000268       __imp__HeapFree@12         10057268     kernel32:KERNEL32.dll
 0004:0000026c       __imp__DisableThreadLibraryCalls@4 1005726c     kernel32:KERNEL32.dll
 0004:00000270       __imp__FatalAppExitA@8     10057270     kernel32:KERNEL32.dll
 0004:00000274       __imp__GetSystemTimeAsFileTime@4 10057274     kernel32:KERNEL32.dll
 0004:00000278       __imp__MultiByteToWideChar@24 10057278     kernel32:KERNEL32.dll
 0004:0000027c       \177KERNEL32_NULL_THUNK_DATA 1005727c     kernel32:KERNEL32.dll
 0004:000002bc       __imp_?_Unlock@?$basic_streambuf@DU?$char_traits@D@std@@@std@@QAEXXZ 100572bc     msvcprtd:MSVCP80D.dll
 0004:000002c0       __imp_?_Lock@?$basic_streambuf@DU?$char_traits@D@std@@@std@@QAEXXZ 100572c0     msvcprtd:MSVCP80D.dll
 0004:000002c4       __imp_?uncaught_exception@std@@YA_NXZ 100572c4     msvcprtd:MSVCP80D.dll
 0004:000002c8       __imp_?_Osfx@?$basic_ostream@DU?$char_traits@D@std@@@std@@QAEXXZ 100572c8     msvcprtd:MSVCP80D.dll
 0004:000002cc       __imp_?good@ios_base@std@@QBE_NXZ 100572cc     msvcprtd:MSVCP80D.dll
 0004:000002d0       __imp_??6?$basic_ostream@DU?$char_traits@D@std@@@std@@QAEAAV01@M@Z 100572d0     msvcprtd:MSVCP80D.dll
 0004:000002d4       __imp_?tie@?$basic_ios@DU?$char_traits@D@std@@@std@@QBEPAV?$basic_ostream@DU?$char_traits@D@std@@@2@XZ 100572d4     msvcprtd:MSVCP80D.dll
 0004:000002d8       __imp_?flush@?$basic_ostream@DU?$char_traits@D@std@@@std@@QAEAAV12@XZ 100572d8     msvcprtd:MSVCP80D.dll
 0004:000002dc       __imp_?width@ios_base@std@@QBEHXZ 100572dc     msvcprtd:MSVCP80D.dll
 0004:000002e0       __imp_?flags@ios_base@std@@QBEHXZ 100572e0     msvcprtd:MSVCP80D.dll
 0004:000002e4       __imp_?fill@?$basic_ios@DU?$char_traits@D@std@@@std@@QBEDXZ 100572e4     msvcprtd:MSVCP80D.dll
 0004:000002e8       __imp_?rdbuf@?$basic_ios@DU?$char_traits@D@std@@@std@@QBEPAV?$basic_streambuf@DU?$char_traits@D@std@@@2@XZ 100572e8     msvcprtd:MSVCP80D.dll
 0004:000002ec       __imp_?sputc@?$basic_streambuf@DU?$char_traits@D@std@@@std@@QAEHD@Z 100572ec     msvcprtd:MSVCP80D.dll
 0004:000002f0       __imp_?eof@?$char_traits@D@std@@SAHXZ 100572f0     msvcprtd:MSVCP80D.dll
 0004:000002f4       __imp_?eq_int_type@?$char_traits@D@std@@SA_NABH0@Z 100572f4     msvcprtd:MSVCP80D.dll
 0004:000002f8       __imp_?setstate@?$basic_ios@DU?$char_traits@D@std@@@std@@QAEXH_N@Z 100572f8     msvcprtd:MSVCP80D.dll
 0004:000002fc       __imp_?width@ios_base@std@@QAEHH@Z 100572fc     msvcprtd:MSVCP80D.dll
 0004:00000300       __imp_??5?$basic_istream@DU?$char_traits@D@std@@@std@@QAEAAV01@AAM@Z 10057300     msvcprtd:MSVCP80D.dll
 0004:00000304       \177MSVCP80D_NULL_THUNK_DATA 10057304     msvcprtd:MSVCP80D.dll
 0004:0000033c       __imp___except_handler4_common 1005733c     MSVCRTD:MSVCR80D.dll
 0004:00000340       __imp___onexit             10057340     MSVCRTD:MSVCR80D.dll
 0004:00000344       __imp___lock               10057344     MSVCRTD:MSVCR80D.dll
 0004:00000348       __imp____dllonexit         10057348     MSVCRTD:MSVCR80D.dll
 0004:0000034c       __imp___unlock             1005734c     MSVCRTD:MSVCR80D.dll
 0004:00000350       __imp___crt_debugger_hook  10057350     MSVCRTD:MSVCR80D.dll
 0004:00000354       __imp____CppXcptFilter     10057354     MSVCRTD:MSVCR80D.dll
 0004:00000358       __imp___adjust_fdiv        10057358     MSVCRTD:MSVCR80D.dll
 0004:0000035c       __imp___amsg_exit          1005735c     MSVCRTD:MSVCR80D.dll
 0004:00000360       __imp___initterm_e         10057360     MSVCRTD:MSVCR80D.dll
 0004:00000364       __imp___initterm           10057364     MSVCRTD:MSVCR80D.dll
 0004:00000368       __imp___CrtSetCheckCount   10057368     MSVCRTD:MSVCR80D.dll
 0004:0000036c       __imp___decode_pointer     1005736c     MSVCRTD:MSVCR80D.dll
 0004:00000370       __imp___free_dbg           10057370     MSVCRTD:MSVCR80D.dll
 0004:00000374       __imp___encoded_null       10057374     MSVCRTD:MSVCR80D.dll
 0004:00000378       __imp___malloc_dbg         10057378     MSVCRTD:MSVCR80D.dll
 0004:0000037c       __imp___encode_pointer     1005737c     MSVCRTD:MSVCR80D.dll
 0004:00000380       __imp___CRT_RTC_INITW      10057380     MSVCRTD:MSVCR80D.dll
 0004:00000384       __imp____CxxFrameHandler3  10057384     MSVCRTD:MSVCR80D.dll
 0004:00000388       __imp____clean_type_info_names_internal 10057388     MSVCRTD:MSVCR80D.dll
 0004:0000038c       \177MSVCR80D_NULL_THUNK_DATA 1005738c     MSVCRTD:MSVCR80D.dll

 entry point at        0001:00001580


 Exports

  ordinal    name

        1    ?_eLut@@3PAGA (unsigned short * _eLut)
        2    ?_toFloat@@3PATuif@half@@A (union half::uif * _toFloat)
